:1000000008308A0000280000D3346D38EC32202AF2
:10001000E832F236EF36653AE8327210A0060A008E
:10002000D43270366F3A6110753BEE347439A034B7
:100030006F1DA0124C32A0210D050000CE30F03211
:10004000F434A031EC30EE35751DA0124C32A036E0
:1000500056100D0500015039EF3A641DA0124C32C4
:10006000A03641100D050001CB30F030E334F43000
:10007000203DE23CF4326B1DA0124C32A0364134DC
:100080000D050001CB30F030E334F430A036613C94
:100090003A1025266410ED20E8060A00533A613B29
:1000A0003A10252664102838F237E3326E3AE1140C
:1000B0000D050000A0132008831687008312871304
:1000C0000830F80063280000F8177428F813C20CF1
:1000D00003188717031C8713781774287813F80BF5
:1000E00067287228000087173F308400840B762829
:1000F0000000F81B6628781B6E280800831603177B
:100100008C170C140000000083120C087F390319AF
:10011000C2280313B90003170D080313BA0003170D
:100120000F080313BB003908C2005A203A0803170E
:100130008D0003133B0803178F0083168C170C14D4
:100140000000000083120C0D0E0D7F390319C22828
:100150000313B90003170D080313BA0003170F08A0
:100160000313BB003908C2005A203A0803178D0058
:1001700003133B0803178F008D0A03198F0A03131B
:100180007E28031703138A150A126D280830F80019
:1001900000008711A0112008831687000000831239
:1001A000B90D0712031CDA282016200883168700D1
:1001B000DE28831220122008831687000000831295
:1001C000A0152008831687008312871DE528F80BE9
:1001D000C82800008711A01120088316870000009E
:1001E0008312201620088316870000000000831267
:1001F000A0152008831687008312871DFD28F801AB
:100200000000071A78148711A011200883168700B0
:100210008312071220122008831687008312080019
:100220000830BA007708BB00201620088316870024
:1002300000008312A0152008831687008312871DF3
:100240001F29071A0314071E0310F80D0000A01140
:1002500020088316870083128711BA0B14292016F1
:100260002008831687000000831207123B08031939
:100270003E29201220088316870083120000A01553
:100280002008831687008312871D442900008711E8
:10029000A011200883168700000083120712201285
:1002A00020088316870083120800F801F901F7017E
:1002B000FA013C08031D5F293B0803197929103016
:1002C000BD000310B90DBA0DF70DFA0D3C087A0206
:1002D000031D6C293B087702031C75293B08F702B4
:1002E000031CFA033C08FA020314F80DF90DBD0BC8
:1002F00061298A150A12BF2D831603178C170C1457
:10030000000000000318AB2983120C087F39031387
:10031000BA0003170D080313BB0003170F080313DC
:10032000BC003A08C2005A203B0803178D00031393
:100330003C0803178F0083168C170C140000000074
:1003400083120313B90BA529A82983160317AB2918
:10035000CA298316031783120C0D0E0D7F39031360
:10036000BA0003170D080313BB0003170F0803138C
:10037000BC003A08C2005A203B0803178D00031343
:100380003C0803178F008D0A03198F0A031003130B
:10039000B90B7C290800C1010408C0004110831B6F
:1003A0004114BA1FDB29C017401EC00AB909BA0997
:1003B000B90A0319BA0A3A0EF038BC00BC07E23E8B
:1003C000BD00323EBF003A080F39BD07BD07BF0769
:1003D000E93EBE00BE07BE07390E0F39BE07BF0794
:1003E000BE0DBF0DBF09BF0D39080F39BF07BC0DCA
:1003F0000730BB000A30BF07BE03031CFB29BE0742
:10040000BD03031CFF29BD07BC03031C032ABC0753
:10041000BB03031C072A3B308400831307304005CD
:10042000401384034005031D1C2A401A840A401A05
:100430001C2A2030F700392A84073F3004020319B0
:1004400040170008F700031D2D2A401B2D2A401AD3
:10045000472AC0192D2A2030382AC01F352A2D30AE
:10046000F70084034013C013392AC01540123030FE
:10047000F707BA010408B9003A10831B3A14770849
:10048000C2005A203908840083133A188317840A5B
:10049000401F1D2A08003A30840083130008031906
:1004A0005E2A0230F800F701F70B542AF80B532AA2
:1004B0009730F700F70B5A2A800B512A8A150A1237
:0204C000D52E37
:10100000840183131F308305713083168F000F080E
:101010008312A01320088316870083128717831674
:1010200003170908C039890003131F129F120030EB
:10103000031788008312870188018901FF30031399
:10104000A000831603170908C039890003131F1273
:101050009F12003003178800831203131F139F137E
:1010600083169F1383121F149412A0122008831654
:101070008700831220162008831687008312A01190
:1010800020088316870001308312940000308316F5
:1010900094000108C739083881008312900100309C
:1010A000F800920000308316920083122015200869
:1010B000831687008312970183169B019C010130E0
:1010C0009D008312031787018801890104308D0078
:1010D00000308F008A1103137E288A1520162008FD
:1010E0008316870000008312A0152008831687004E
:1010F00000008312071220122008831687000000C8
:1011000083128711A011200883168700AA3083124A
:10111000B9008A11C6208A150C30B9008A11C62080
:101120008A15201620088316870000008312A01558
:1011300020088316870000008312871D9D28071250
:101140002012200883168700000083128711A01147
:10115000200883168700AB308312B9008A11C6209D
:101160008A15F7018A1110218A157808A10020122A
:1011700020088316870000008312A015200883161C
:1011800087008312871DC2280000C6280000201691
:10119000200883168700000083122016200883167B
:1011A000870000008312A015200883168700000026
:1011B0008312071220122008831687000000831272
:1011C0008711A011200883168700AA308312B90066
:1011D0008A11C6208A150D30B9008A11C6208A15D9
:1011E000201620088316870000008312A01520080F
:1011F0008316870000008312871DFC280712201227
:10120000200883168700000083128711A011200890
:1012100083168700AB308312B9008A11C6208A1565
:10122000F7018A1110218A157808A20020122008DF
:101230008316870000008312A015200883168700FC
:101240008312871D2129000025290000201620086F
:10125000831687000000831220162008831687005B
:1012600000008312A0152008831687000000831257
:1012700007122012200883168700000083128711AE
:10128000A011200883168700AA308312B9008A11A2
:10129000C6208A150830B9008A11C6208A15201286
:1012A00020088316870000008312A01520088316EB
:1012B00087008312871D5A2900005E29000020162E
:1012C000200883168700000083122016200883164A
:1012D000870000008312A0152008831687000000F5
:1012E0008312071220122008831687000000831241
:1012F0008711A011200883168700AB308312B90034
:101300008A11C6208A15F7018A1110218A157808DA
:10131000A300201220088316870000008312A01566
:101320002008831687008312871D942900009829BE
:101330000000201620088316870000008312201664
:1013400020088316870000008312A015200883164A
:1013500087000000831207122012200883168700DE
:10136000000083128711A011200883168700AA307D
:101370008312B9008A11C6208A150930B9008A1172
:10138000C6208A15201220088316870000008312C9
:10139000A0152008831687008312871DCD29000021
:1013A000D129000020162008831687000000831230
:1013B000201620088316870000008312A01520083D
:1013C000831687000000831207122012200883165C
:1013D0008700000083128711A01120088316870060
:1013E000AB308312B9008A11C6208A15F7018A1121
:1013F00010218A157808A40020122008831687007F
:1014000000008312A0152008831687008312871D11
:10141000072A00000B2A00002016200883168700E8
:101420000000831220162008831687000000831214
:10143000A0152008831687000000831207122012CF
:10144000200883168700000083128711A01120084E
:1014500083168700AA308312B9008A11C6208A1524
:101460000A30B9008A11C6208A1520122008831676
:10147000870000008312A0152008831687008312BE
:10148000871D402A0000442A0000201620088316E9
:1014900087000000831220162008831687000000B2
:1014A0008312A015200883168700000083120712FC
:1014B0002012200883168700000083128711A011D4
:1014C000200883168700AB308312B9008A11C6202A
:1014D0008A15F7018A1110218A157808A5002012B3
:1014E00020088316870000008312A01520088316A9
:1014F00087008312871D7A2A00007E2A00002016AA
:101500002008831687000000831220162008831607
:10151000870000008312A0152008831687000000B2
:1015200083120712201220088316870000008312FE
:101530008711A011200883168700AA308312B900F2
:101540008A11C6208A150B30B9008A11C6208A1567
:10155000201220088316870000008312A01520089F
:10156000831687008312871DB32A0000B72A000064
:1015700020162008831687000000831220162008FA
:101580008316870000008312A015200883168700A9
:101590000000831207122012200883168700000023
:1015A00083128711A011200883168700AB308312A5
:1015B000B9008A11C6208A15F7018A1110218A15EF
:1015C0007808A600201220088316870000008312E6
:1015D000A0152008831687008312871DED2A0000BE
:1015E000F12A0000201620088316870000008312CD
:1015F000201620088316870000008312A0152008FB
:101600008316870000008312071220122008831619
:101610008700000083128711A0112008831687001D
:10162000AA308312B9008A11C6208A150430B90085
:101630008A11C6208A152012200883168700000010
:101640008312A0152008831687008312871D262B7E
:1016500000002A2B000020162008831687000000B7
:101660008312201620088316870000008312A0151D
:10167000200883168700000083120712201220081A
:1016800083168700000083128711A011200883169B
:101690008700AB308312B9008A11C6208A15F70182
:1016A0008A1110218A157808A700201220088316B5
:1016B000870000008312A01520088316870083127C
:1016C000871D602B0000642B000020162008831665
:1016D0008700000083122016200883168700000070
:1016E0008312A015200883168700000083120712BA
:1016F0002012200883168700000083128711A01192
:10170000200883168700AA308312B9008A11C620E8
:101710008A150530B9008A11C6208A1520122008C2
:101720008316870000008312A01520088316870007
:101730008312871D992B00009D2B00002016200886
:101740008316870000008312201620088316870066
:1017500000008312A0152008831687000000831262
:1017600007122012200883168700000083128711B9
:10177000A011200883168700AB308312B9008A11AC
:10178000C6208A15F7018A1110218A157808A80049
:10179000201220088316870000008312A01520085D
:1017A000831687008312871DD32B0000D72B0000E0
:1017B00020162008831687000000831220162008B8
:1017C0008316870000008312A01520088316870067
:1017D00000008312071220122008831687000000E1
:1017E00083128711A011200883168700AA30831264
:1017F000B9008A11C6208A150630B9008A11C620A0
:101800008A15201220088316870000008312A01575
:101810002008831687008312871D0C2C0000102CD3
:10182000000020162008831687000000831220166F
:1018300020088316870000008312A0152008831655
:1018400087000000831207122012200883168700E9
:10185000000083128711A011200883168700AB3087
:101860008312B9008A11C6208A15F7018A11102146
:101870008A157808A9002012200883168700000026
:101880008312A0152008831687008312871D462C1B
:1018900000004A2C00002016200883168700000054
:1018A0008312201620088316870000008312A015DB
:1018B00020088316870000008312071220122008D8
:1018C00083168700000083128711A0112008831659
:1018D0008700AA308312B9008A11C6208A15073002
:1018E000B9008A11C6208A152012200883168700A5
:1018F00000008312A0152008831687008312871D1D
:101900007F2C0000832C00002016200883168700FF
:10191000000083122016200883168700000083121F
:10192000A0152008831687000000831207122012DA
:10193000200883168700000083128711A011200859
:1019400083168700AB308312B9008A11C6208A152E
:10195000F7018A1110218A157808AA0020122008A0
:101960008316870000008312A015200883168700C5
:101970008312871DB92C0000BD2C00002016200802
:101980008316870000008312201620088316870024
:1019900000008312A0152008831687000000831220
:1019A0000712201220088316870000008312871177
:1019B000A011200883168700AA308312B9008A116B
:1019C000C6208A150230B9008A11C6208A15201255
:1019D00020088316870000008312A01520088316B4
:1019E00087008312871DF22C0000F62C00002016C1
:1019F0002008831687000000831220162008831613
:101A0000870000008312A0152008831687000000BD
:101A10008312071220122008831687000000831209
:101A20008711A011200883168700AB308312B900FC
:101A30008A11C6208A15F7018A1110218A157808A3
:101A4000AB00201220088316870000008312A01527
:101A50002008831687008312871D2C2D0000302D4F
:101A6000000020162008831687000000831220162D
:101A700020088316870000008312A0152008831613
:101A800087000000831207122012200883168700A7
:101A9000000083128711A011200883168700AA3046
:101AA0008312B9008A11C6208A150330B9008A1141
:101AB000C6208A1520122008831687000000831292
:101AC000A0152008831687008312871D652D00004E
:101AD000692D00002016200883168700000083125D
:101AE000201620088316870000008312A015200806
:101AF0008316870000008312071220122008831625
:101B00008700000083128711A01120088316870028
:101B1000AB308312B9008A11C6208A15F7018A11E9
:101B200010218A157808AC0020122008831687003F
:101B300000008312A0152008831687008312871DDA
:101B40009F2D0000A32D000020162008831687007B
:101B500000008312BA012208B900BA00B9012108B5
:101B60003907AD003A08AE000318AE0A2E08BA00D5
:101B70002D08B900BC010A30BB008A1155298A150D
:101B80007908BA007808B90011303902AD003A0876
:101B9000AE000130031C0230AE02BA012408B900C5
:101BA000BA00B90123083907AF003A08B00003189A
:101BB000B00ABA012608B900BA00B90125083907E8
:101BC000B1003A08B2000318B20ABA012808B900F5
:101BD000BA00B90127083907B3003A08B40003185E
:101BE000B40ABA012A08B900BA00B90129083907AC
:101BF000B5003A08B6000318B60ABA012C08B900B5
:101C0000BA00B9012B083907B7003A08B800031821
:101C1000B80A103003178D0000308F000310133006
:101C20000313B9008A117C218A15103084002E0814
:101C3000BA002D08B9008A11CB218A151B30031771
:101C40008D0000308F00031004300313B9008A1197
:101C50007C218A151E3003178D0000308F00031081
:101C60000F300313B9008A117C218A1510308400CB
:101C70003008BA002F08B9008A11CB218A15273005
:101C800003178D0000308F00031006300313B900D6
:101C90008A117C218A152B3003178D0000308F00AC
:101CA000031007300313B9008A117C218A15103004
:101CB00084003208BA003108B9008A11CB218A1594
:101CC000303003178D0000308F00031006300313EF
:101CD000B9008A117C218A15343003178D00003039
:101CE0008F00031011300313B9008A117C218A156B
:101CF000103084003408BA003308B9008A11CB21AF
:101D00008A153E3003178D0000308F000310063017
:101D10000313B9008A117C218A15423003178D0004
:101D200000308F0003100E300313B9008A117C219C
:101D30008A15103084003608BA003508B9008A11B7
:101D4000CB218A154A3003178D0000308F00031411
:101D500006300313B9008A117C218A154E3003170F
:101D60008D0000308F00031006300313B9008A1174
:101D70007C218A15103084003808BA003708B90071
:101D80008A11CB218A15523003178D0000308F0045
:101D900003140D300313B9008A117C218A15083011
:101DA000B900FA30BA008A114B2A8A15B90BD12E24
:041DB0006E28630036
:04400E00F52CFF3F4F
:00000001FF
